:100003004E4F4B49412033353130492D00474F4F37
:1000130044004C43440000000000000000000000C6
:1000230000000000202020202020002000000028C5
:100033005050000000000000000000002828FC28A9
:1000430050FC50500000002078A8A0603028A8F091
:100053002000000048A8B050283454480000000095
:1000630020505078A8A8906C000000404080000009
:100073000000000000000004081010101010100809
:100083000400004020101010101010204000000049
:100093000020A87070A8200000000000202020F895
:1000A30020202000000000000000000000000040AD
:1000B30040800000000000F8000000000000000085
:1000C3000000000000000040000000081010102095
:1000D30020404040800000007088888888888870AD
:1000E300000000002060202020202070000000007D
:1000F30070888810204080F8000000007088083065
:1001030008088870000000001030505090781018D4
:1001130000000000F88080F00808887000000000EC
:10012300709080F08888887000000000F89010209C
:100133002020202000000000708888708888887044
:10014300000000007088888878084870000000006C
:10015300000020000000002000000000000000203C
:100163000000002020000004081020402010080494
:10017300000000000000F80000F80000000000404C
:100183002010080408102040000000007088881028
:100193002020002000000000708898A8A8B880786C
:1001A3000000000020203050507848CC00000000B0
:1001B300F0484870484848F0000000007888808084
:1001C3008080887000000000F0484848484848F0A4
:1001D30000000000F8485070504048F8000000004C
:1001E300F8485070504040E00000000038488080DC
:1001F3009C88483000000000CC484878484848CCE8
:1002030000000000F8202020202020F8000000003B
:100213007C10101010101090E0000000EC485060AB
:10022300505048EC00000000E0404040404044FC97
:1002330000000000D8D8D8D8A8A8A8A800000000BB
:10024300DC486868585848E80000000070888888CF
:100253008888887000000000F0484870404040E003
:10026300000000007088888888E8987018000000F3
:10027300F0484870504848EC0000000078888060DF
:10028300100888F000000000F8A82020202020702B
:1002930000000000CC4848484848483000000000AF
:1002A300CC4848505030202000000000A8A8A87077
:1002B3005050505000000000D8505020205050D8CB
:1002C30000000000D85050202020207000000000C3
:1002D300F8901020204048F800000038202020200B
:1002E300202020203800004040402020101010081B
:1002F300000000701010101010101010700000207B
:10030300500000000000000000000000000000009A
:100313000000000000FC00200000000000000000BE
:1003230000000000000000304838483C0000000096
:10033300C04040704848487000000000000000388A
:100343004840403800000000180808384848483C36
:100353000000000000000030487840380000000032
:100363001C20207820202078000000000000003CA2
:100373004830407844380000C0404070484848EC5A
:10038300000000002000006020202070000000001A
:10039300100000301010101010E00000C040405C4E
:1003A300507048EC00000000E0202020202020F8BE
:1003B30000000000000000F0A8A8A8A800000000AA
:1003C300000000F0484848EC000000000000003046
:1003D3004848483000000000000000F048484870DA
:1003E30040E000000000003848484838081C00007E
:1003F300000000D8604040E00000000000000078EA
:1004030040300878000000000020207020202018D1
:1004130000000000000000D84848483C00000000ED
:10042300000000EC4850302000000000000000A84D
:10043300A870505000000000000000D8502050D891
:1004430000000000000000EC4850302020C00000F5
:1004530000000078102020780000001810101020F1
:100463001010101018001010101010101010101091
:10047300101000602020201020202020600040A4C5
:1004830018000000000000000000004FFE0407FCFD
:1004930066455444466455444445C0000407FC0083
:1004A30001F8108FFE8023F80400401C00000400B4
:1004B300447FE4447FC4444447FC44004203E000D7
:1004C3007FC008010060044FFE0400400400401C8C
:1004D30000000A8F24120FFE1201643A8D101321BB
:1004E300CA7060001F81081F81081F8000FFE2405F
:1004F30037C4C087E000040060090108246C40177A
:100503008140140140FFE000308DBC524FB452C70C
:1005130060DBE5026BE4A2C6C0000A8F24120FFE63
:100523001201643A8D101321CA7060002102202742
:10053300EB42AC2A4227E24224224227E000450252
:10054300480FE0C8D7E44844847E54867E04000004
:100553000000000000000000000000000000000098
:100563000000FFFFFFFFFFFFFFFFFFFFFFFFFFFF96
:10057300FFFFFFFFFFFFFFFFFFFFFFFFFFFFFFFF88
:10058300FFFFFFFFFFFFFFFFFFFFFFFFFFFFFFFF78
:10059300FFFFFFFFFFFFFFFFFFDB926D45242424D6
:1005A300244992B6FFFFFFFFFFFFFFFFFFFFFFFF9F
:1005B300FFFFFFFFFFFFFFFFFFFFFFFFFFFFFFDB6C
:1005C3006D24002424242424242400004992DBFFE6
:1005D300FFFFFFFFFFFFFFFFFFFFFFFFFFFFFFFF28
:1005E300FFFFFFFFFFFF9224002424242424494516
:1005F30024242424000024B6FFFFFFFFFFFFFFFF96
:10060300FFFFFFFFFFFFFFFFFFFFFFFFFF6D002463
:1006130024494924494949494924242424240000DC
:1006230092FFFFFFFFFFFFFFFFFFFFFFFFFFFFFF44
:10063300FFFFFFFF920024244949496D4949494975
:1006430049494924242424000092FFFFFFFFFFFFB0
:10065300FFFFFFFFFFFFFFFFFFFFFFB62424244937
:100663004949B6FFB64949496DDBB64924242424D8
:100673000024DBFFFFFFFFFFFFFFFFFFFFFFFFFF85
:10068300FFFFFF49002449494992FFFFFF9249496F
:10069300DBFFFFB62424242424006DFFFFFFFFFFAC
:1006A300FFFFFFFFFFFFFFFFFFFF920024494949C0
:1006B30049B6FFDB92924992DB6DFFDB4924242488
:1006C300240024DBFFFFFFFFFFFFFFFFFFFFFFFF10
:1006D300FFFF6D002449494949DBFFB6004949B68C
:1006E300926D6DFF6D24242424000092FFFFFFFF11
:1006F300FFFFFFFFFFFFFFFFFFDB242424494949DE
:1007030049B6FFDB49924992FFFFFFDB49242424CA
:1007130024240049DBFFFFFFFFFFFFFFFFFFFFFF75
:10072300FFB62024494949494992FFFFFF922449D2
:10073300FFFFFFDB2424242424240024DBFFFFFF0A
:10074300FFFFFFFFFFFFFFFFFF92002449494949D5
:100753004949B6DB9649252572DBBB6D2424242445
:1007630024240024B6FFFFFFFFFFFFFFFFFFFFFF6F
:10077300FF4D0424494949494949496D686C8C8CAA
:10078300686D4924252424242424000092FFFFFFBC
:10079300FFFFFFFFFFFFFFFFDB6444244949494993
:1007A3008DADD0D0F0F4F4F4F0F0CCAC8848242430
:1007B3002424000049DBFFFFFFFFFFFFFFFFFFFFD4
:1007C3008DA0A024294988CCF5FAF4F4F4F4F4F4C8
:1007D300F4F4F0F0F0EC8824240420404096FFFF6A
:1007E300FFFFFFFFFFFFFFFFA4A0E0A04449ACF021
:1007F300F0F5F4F4F4F4F4F4F4F4F0F0F0F0AC24E1
:10080300044080804092FFFFFFFFFFFFFFFFFFFFD9
:10081300C4C0C4E4C06449496868D0F0F4F4F4F493
:10082300F4F0D0884848242460A080804496FFFFD9
:10083300FFFFFFFFFFFFFF6D60E0E0EDE9E0A06475
:10084300444529688CB0B0B08C682424244460A04B
:10085300C0A0A0600092FFFFFFFFFFFFFFFF6D003E
:100863002484E0E0E9EDE9E4E0A0846464444444E2
:1008730044446060A0C0C0C0A0A080200024DBFF6F
:10088300FFFFFFFFFF920020242484E0E0E4E9E47B
:10089300E0E0E0E0E0E0C0C0C0C0E0E0E0E0C0A035
:1008A300A060200000006DFFFFFFFFFFDB000024BE
:1008B300242492FBC9C0E0E0E0E0E0E0E0E0E0E017
:1008C300E0E0E0E0E0C0A084B2490000000024B60C
:1008D300FFFFFFFF6D0024242449DBFFDBA4C0C01E
:1008E300C0E0E0E0E0E0E0E0E0E0E0C0A08992BB4F
:1008F300DBB624000000006DFFFFFFB600002424D8
:10090300246DFFFFD7C4E0C080A0A4C4C4C0C0C08E
:10091300C4C4A98DB6DBDFDBDBDB6D000000002484
:10092300DBFFFF92000024242492FFFFD6E9E0E0DE
:10093300A0A0B2FBDBD6D6D6DBDBDFFFFFFFDBDB22
:10094300DBDB920000000000B6FFFF490000242417
:100953002492FFFFD2E9E4E0C0E0D2FFFFFFFFFFF4
:10096300FFFFFFFFFFDBDBDBDBDBB600000000008C
:1009730092FFFF24000020242492FFFFD6E4E0E04E
:10098300E0E0D2FFFFFFFFFFFFFFFFFFFFDBDBDB4B
:10099300DBDBB6000000000092FFFF2400002424EC
:1009A300006DFFFFDBC4E0E0E0C0D2FFFFFFFFFF0D
:1009B300FFFFFFFFFFDBDBDBDBDB92000000000060
:1009C30092FFFF4900246D6D0024DBFFFFD689A44D
:1009D300A4A9DBFFFFFFFFFFFFFFFFFFFFDBDBDB65
:1009E300DBDB6D006D24000092FFFFB6496DDBDB9E
:1009F300240092FFFFFFDFDBDBDFFFFFFFFFFFFFD3
:100A0300FFFFFFFFFFDBDBDBDBDB2424B6920049C8
:100A1300B6FFFFFFDBDBFFFF920049DBFFFFFFFFBA
:100A2300FFFFFFFFFFFFFFFFFFFFFFFFDBDBDBDB63
:100A3300DB6D006DDBFFDBB6DBFFFFFFFFFFFFFFBF
:100A4300FF920049FFFFFFFFFFFFFFFFFFFFFFFFD5
:100A5300FFFFFFDBDBDBDBDB920049B6FFFFFFFFC2
:100A6300FFFFFFFFFFFFFFFFFFB6882049DBFFFF0C
:100A7300FFFFFFFFFFFFFFFFFFFFDBDBDBDBDB92A4
:100A830024688DB6FFFFFFFFFFFFFFFFFFFFFFDBC4
:100A9300ADCCF0AC4449B7FFFFFFFFFFFFFFFFFF03
:100AA300FFDBDBDBDBDB6E44B0F4D068B6FFFFFFBC
:100AB300FFFFFFFFFFFFFF9288F0F0F0F08C486923
:100AC300B6DBFFFFFFFFFFFFFFDFDBBB926888F0B2
:100AD300F4F4F4D08CB6FFFFFFFFFFFFFFFFFF919D
:100AE300CCF0F0F0F4F4F0AC886891B6B6B6B6B6D4
:100AF300B6B6B28C88CCF4F4F4F4F4F48C6EFFFF45
:100B0300FFFFFFFFFFFFFFDBACECF0F0F0F4F4F4CA
:100B1300F4F0D08824496D6D4988ACCCF0F4F4F43A
:100B2300F4F4F48C6992FFFFFFFFFFFFFFFFFFFF69
:100B3300DA8D8CACCCCCD0D0ACAC8C686D92B6B624
:100B4300928D8C8CACACACACAC8C6C6D92DBFFFF3F
:100B5300FFFFFFFFFFFFFFFFFFDBB6B6929292920C
:100B630092929296DBFFFFFFFFFFDBB6B6B2929243
:100B73009292B6DBFFFFFFFFFFFFFFFFFFFFFFFFC9
:100B8300FFFFFFFFFFFFFFFFFFFFFFFFFFFFFFFF72
:100B9300FFFFFFFFFFFFFFFFFFFFFFFFFFFFFFFF62
:020BA300FFFF52
:0311EC00011F419F
:0711C5001211067F057E00F8
:1011CC00E4FDFCC3ED9FEC9E5015E4FBFA0BBB0059
:0F11DC00010AEB64644A70F50DBD00010C80E45C
:0111EB0022E1
:1010E1007FFF1211067FFD1211067FFC1211067F90
:1010F100FB1211067FFA1211067FF91211067FF712
:051101001211067FF051
:10110600C2A0C2A4ED7004C2A38002D2A3D2A4E4FA
:10111600FEC2A4EF30E704D2A38002C2A3EF25E00B
:09112600FFD2A40EBE08EAD2A01B
:01112F00229D
:10100700E4FD7F09121106C2A0C2A4E4FF74082FF1
:10101700F8E4F6FED2A420A318C374079EFD74015A
:10102700A805088002C333D8FCFD74082FF8E64DE5
:10103700F6C2A40EBE08DD0FBF06D2E50860122473
:1010470081600924807025751F418020751F4280AB
:101057001BE509250AFFE433FE7C00EF250BFFECB7
:0E1067003E4F7005751F448003751F43D2A0D5
:011075002258
:100CD600D2A1D2A0C2A3D2A4C2A17F327E00121199
:100CE600CCD2A11211CCE4FDFF1211C5E4FD7F01A7
:100CF6001211C5E4FD7FC61211067FB91211060D49
:100D0600E4FF121106121007E4FD7FB51211060D5D
:100D16007F011211061D7FBD121106E51FB44405A1
:100D26000D7F0480047D01E4FF121106E4FD7FBE01
:100D36001211060D7F031211061D7F111211067F77
:100D4600BA1211060D7F7F1211067F031211061DBE
:100D56007F36121106E51FB441050D7F0880047D1C
:100D660001E4FF121106E4FD7FB7121106E4FC7DD3
:100D760001E4FF1211060CBC0EF5E4FD7F291211E9
:100D8600067F031211067F147E001211CCE4FD7F4C
:100D9600201211067F25121106E51F24BE601014CD
:100DA6006013146016240370197D017F4680107D40
:100DB600017F43800A7D017F4280047D017F3112DD
:020DC600110614
:010DC8002208
:100DC900BF010DE4FD7F3A1211060D7F03020E7675
:100DD900E4FD7F3A1211060D7F021211061D7F2DC7
:100DE900121106E51F64426006E51F6443701B7D0E
:100DF900011210E11210E17FFF1211067FFC12119E
:100E0900067FF91211067FF080637D01E4FF12115C
:100E1900067F021211067F031211067F04121106C2
:100E29007F051211067F061211067F081211067F2F
:100E39000F121106E4FF1211067F021211067F0339
:100E49001211067F041211067F051211067F061280
:100E590011067F081211067F0F121106E4FF121105
:100E6900067F031211067F061211067F0F12110663
:010E79002256
:06116700FBED240BF51E58
:10116D00AC07AA05E4FD7F2A121106AF040D12117A
:10117D0006AF031211061D7F2B121106AF020D12C1
:0D118D001106AF1E1211061D7F2C02110667
:061076008E088F098D0AAF
:10107C00751E427B61E4FDFF12116DE50A6401707F
:10108C003AF50BE4F9E508C4F854F0C8E509C45482
:10109C000F48FF7D01121106E508FFE509540FFE0C
:1010AC00C454F04FFF121106AF0912110609B931E1
:1010BC00D4050BE50BC3944340C922E4F50BE4F9CA
:1010CC00AF097D0112110609B962F5050BE50BC3D9
:0410DC00944340EA0F
:0110E00022ED
:020F06008B134B
:100F08007518FF751900751A19EF2407121167E58E
:100F18001324E0FFE434FFFE7C007D0C1211B3EFD4
:100F2800251AF51AEE3519F519E4F517E4F516AB97
:100F380018AA19A91A12119AFD7C00C374079516EC
:100F4800FF74017E00A807088005C333CE33CED8CE
:100F5800F9FFEE5CFEEF5D4E7D016004AF14800288
:100F6800AF151211060516E516C3940840C17401A1
:100F7800251AF51AE43519F5190517E517C3940C60
:020F880040AA7D
:010F8A002244
:061130008B0A8A0B890CFA
:101136008F0F8D10AB0AAA0BA90C12119AFB602017
:10114600850D14850E15AD10AF0F120F0674072509
:101156000FF50F7401250CF50CE4350BF50B80D457
:011166002266
:020F8B008B0ACF
:100F8D00750FFF75100475118DEF240B121167E5A8
:100F9D000A75F012A4AEF02511F511EE3510F5100D
:100FAD00E4F50EE4F50DAB0FAA10A91112119AFD7F
:100FBD007C00C37407950DFF74017E00A80708809F
:100FCD0005C333CE33CED8F9FFEE5CFEEF5D4E7D1B
:100FDD00016004AF0B8002AF0C121106050DE50D7B
:100FED00C3940840C174012511F511E43510F510B5
:090FFD00050EE50EC3941240AA92
:0110060022C7
:100BA500120CD6E4FF120DC9E4FD7FFFFE1210768C
:100BB500751E277B43E4FD7F1C12116DE4FBFA745F
:100BC500652BF58274053AF583E493FF7D011211D7
:100BD500060BBB00010ABA06E6BB40E3750BE075E0
:100BE5000CFF7B047D28E4FF120F8B750BE0750C61
:100BF500FF7B057D287F0E120F8B750BE0750CFFB3
:100C05007B067D287F1C120F8B750BE0750CFF7B17
:100C1500077D287F2A120F8B750BE0750CFF7B086B
:100C25007D287F38120F8B750BE0750CFF7B097DD6
:100C3500287F46120F8B750BE0750CFF7B0A7D280C
:100C45007F54120F8B750B03750CFFE4FB7D05FFBD
:100C5500120F8B750B03750CFF7B017D057F0E1243
:100C65000F8B750B03750CFF7B027D13E4FF120FD1
:100C75008B750B03750CFF7B037D137F0E120F8B9A
:100C85007BFF7A007903750D03750EFF7D377F05B0
:100C95001211307514037515FFAB1F7D377F5A127E
:100CA5000F067BFF7A007910E4F50D750EFF7D05C3
:100CB5007F441211307BFF7A007915E4F50D750E2E
:100CC500FF7D117F4B1211307FDC7E051211CC8028
:010CD500F727
:03000000020E7A73
:0C0E7A00787FE4F6D8FD75811F020EC1E0
:10119A00BB010689828A83E0225002E722BBFE0253
:0911AA00E32289828A83E4932286
:1011B300EF8DF0A4A8F0CF8CF0A428CE8DF0A42E50
:0211C300FE220A
:100E8600020BA5E493A3F8E493A34003F68001F2D2
:100E960008DFF48029E493A3F85407240CC8C3336D
:100EA600C4540F4420C8834004F456800146F6DF3C
:100EB600E4800B01020408102040809011ECE47ECF
:100EC600019360BCA3FF543F30E509541FFEE49331
:100ED600A360010ECF54C025E060A840B8E493A3F8
:100EE600FAE493A3F8E493A3C8C582C8CAC583CA23
:100EF600F0A3C8C582C8CAC583CADFE9DEE780BEDB
:0111EF0000FF
:00000001FF
